:041800000CEF0CF0ED
:10180800FACF2BF0FBCF2CF0E9CF2DF0B2ED18F08A
:1018180047EF1AF08C0F8C0F020104FC0300140030
:10251C000102FC0328C408F51200A6A21200FDD784
:10252C00010E69EC1EF01200020E69EC1EF0120096
:10253C00020E38EC1FF01200D6CF03F0D7CF04F008
:10254C0003C001F004C002F0120001C0A9FFA69C58
:10255C00A69EA68000F000F0A8501200D6CF62F024
:10256C00D7CF63F062C060F063C061F0120060C04E
:10257C00A9FFA69CA69EA68000F000F0A850120011
:10258C000001606F010E0001F26F60C0F1F00201FA
:10259C0000511200016E01507F0BD56E000ED76EEC
:1025AC00000ED66EF29401AE02D0F28A01D0F29AED
:1025BC00D58E1200000E026E000E016EABEC12F006
:1025CC000001E66F040E0001E66503D0000E000169
:1025DC00E66F12000001E651050D590EF3240001BF
:1025EC00616F7F0EF4200001626F050E0001636FB6
:1025FC005FEC17F012000001EA51040D860EF32473
:10260C000001616F7F0EF4200001626F040E000167
:10261C00636F5FEC17F012000001EC51050D9A0E80
:10262C00F3240001616F7F0EF4200001626F050E30
:10263C000001636F5FEC17F012000001F051060D02
:10264C00B70EF3240001616F7E0EF4200001626F5F
:10265C00060E0001636F5FEC17F012000001E551EC
:10266C00040D230EF3240001616F7F0EF420000192
:10267C00626F040E0001636F5FEC17F01200000133
:10268C00EF51060DDB0EF3240001616F7E0EF4207A
:10269C000001626F060E0001636F5FEC17F0120011
:1026AC000001F351050DFD0EF3240001616F7D0E49
:1026BC00F4200001626F050E0001636F5FEC17F0F0
:1026CC0012000001F451040DCC0EF3240001616FD3
:1026DC007F0EF4200001626F040E0001636F5FEC4B
:1026EC0017F01200000E0001616F000E0001606F08
:1026FC00BDEC12F00001E66F040E0001E66503D09C
:10270C00000E0001E66F1200010E0001606F000167
:10271C00E651030AD8B408D00001E651040AD8B433
:10272C0003D0000E0001606F00016051120069843B
:10273C0068986D82010E0001E86F000E166E750E22
:10274C00156E000E186E000E176E000E1A6E000E2F
:10275C00196E7CEC18F012000001F1510001F25DD1
:10276C00D8A002D0000E0CD00001F251010D0201D4
:10277C00000EF324D96E0201020EF420DA6EDF5043
:10278C00120002C008F001C007F008D007C0D9FF42
:10279C0008C0DAFF03C0DFFF074A082A0506D8A0E5
:1027AC0006060528D8B40628D8B41200EFD70401C1
:1027BC00040E0001D26F0401280E0001D16F000E2F
:1027CC000001D66F080E0001D56F250E0001D86FE1
:1027DC00200E0001D76F0001D48F12000001E62BF0
:1027EC00040E0001E66503D0000E0001E66F93ECC9
:1027FC0012F0000E0001616F000E0001606FE6C068
:10280C0062F0B0EC15F0F0EC12F012000001EA2BC3
:10281C00040E0001EA6503D0000E0001EA6F93EC90
:10282C0012F0000E0001616F030E0001606FEAC030
:10283C0062F0B0EC15F001EC13F012000001EC2B7F
:10284C00030E0001EC6503D0000E0001EC6F93EC5D
:10285C0012F0000E0001616F060E0001606FECC0FB
:10286C0062F0B0EC15F012EC13F012000001F02B3A
:10287C00050E0001F06503D0000E0001F06F93EC23
:10288C0012F0000E0001616F010E0001606FF0C0CC
:10289C0062F0B0EC15F023EC13F012000001E52B04
:1028AC00060E0001E56503D0000E0001E56F93EC08
:1028BC0012F0000E0001616F050E0001606FE5C0A3
:1028CC0062F0B0EC15F034EC13F012000001EF2BB9
:1028DC00050E0001EF6503D0000E0001EF6F93ECC5
:1028EC0012F0000E0001616F040E0001606FEFC06A
:1028FC0062F0B0EC15F045EC13F012000001F32B74
:10290C00070E0001F36503D0000E0001F36F93EC8A
:10291C0012F0000E0001616F020E0001606FF3C037
:10292C0062F0B0EC15F056EC13F012000001F4510B
:10293C00D8A402D0010E01D0000E0001F46F93EC6C
:10294C0012F0000E0001616F080E0001606FF4C000
:10295C0062F0B0EC15F067EC13F012000001E967BF
:10296C0015D0000E6D6E000E696E160E6F6E9F0EFA
:10297C006B6E7B0E696ED08EA28AA08AF28E01D00D
:10298C006D866DA6FDD7010E0001E96F12000001E6
:10299C0061516011D8A402D0270E12D000016151F0
:1029AC006011D8B40CD00A0E0001605D000E00015D
:1029BC006159D8B004D0000160511D0F01D02C0E0C
:1029CC0012000001685100016A03F3CF6CF0F4CFE0
:1029DC006DF00001685100016B03F35000016D278D
:1029EC000001695100016A03F35000016D276CC0AE
:1029FC0068F06DC069F01200000E0001E86F000E67
:102A0C00166E740E156E000E186E000E176E000EFC
:102A1C001A6E000E196E7CEC18F06D92699468B801
:102A2C0069A803D0689801D0689468A41200FCD7F8
:102A3C00000161C067F0000160C066F00AD066C09A
:102A4C00D9FF67C0DAFF000162C0DFFF0001664BEF
:102A5C00672B00016407D8A0650700016429D8B46E
:102A6C006529D8B41200EBD7000E0001636F00018A
:102A7C00ED51D8B413D060C0D9FF61C0DAFFDF507C
:102A8C000001626FDD0E00016217D8A407D00001AF
:102A9C00F051D8B403D0010E0001636F00016351F3
:102AAC0012000001646FFE0EF66E170EF76E090031
:102ABC00F5CF62F00900F5CF63F0020E0001625D04
:102ACC00000E6359D8A005D000016451B8EC17F082
:102ADC0004D00001645110EC16F012000001646F78
:102AEC00FE0EF66E170EF76E0900F5CF62F00900B8
:102AFC00F5CF63F0020E0001625D000E6359D8A0A1
:102B0C0005D00001645110EC16F004D000016451A2
:102B1C00B8EC17F0120070A01BD0800E39C0D9FF92
:102B2C003AC0DAFFDF6213D0840ED9C0D9FFDAC005
:102B3C00DAFFDF620CD039C0D9FF3AC0DAFF0C0ED5
:102B4C00DF6E39C0D9FF3AC0DAFF000EDB8E709011
:102B5C00689A1200000E0001636F60C0A9FF62C08A
:102B6C00A8FFA69EA69CA684000EF2BE010E000134
:102B7C00636FF29E550EA76EAA0EA76EA682A6B222
:102B8C00FED7000163B102D0F29E01D0F28EA69462
:102B9C0012006DA217D0010E57EC15F0020E57EC77
:102BAC0015F0030E57EC15F013D09CEC16F010D06A
:102BBC00010E74EC15F0020E74EC15F0030E74ECAF
:102BCC0015F006D00001E951200AD8B4EED7F0D7A1
:102BDC001200000E38EC1FF00EEC17F0A5EC29F0EB
:102BEC00B4EC14F0CFEC15F0200E0001E95DD8A088
:102BFC00F9D76DA208D0B1EC19F00009D8B4F2D70E
:102C0C0032EC16F0EFD70001E851D8A4EBD72FEC3B
:102C1C0033F0E8D70001606F13D057C0D9FF58C00C
:102C2C00DAFF5B500BD059C0D9FF5AC0DAFF5C50A9
:102C3C0005D094C1D9FF95C1DAFF5D50DF120BD0DE
:102C4C0000016051010AD8B4E8D7030AD8B4EBD715
:102C5C00010AD8B4EED712000001E751D8B41DD048
:102C6C000001E851D8B419D0A09A9EEC12F06D92E4
:102C7C00180E00016B6F5F0EE82EFED76B2FFCD782
:102C8C0000F06D84100E00016B6F940EE82EFED7D1
:102C9C006B2FFCD700D06D94A08A12000E6E09A485
:102CAC0005D0000E016E0E5094EC1AF009A205D05E
:102CBC00010E016E0E5094EC1AF00E50010D700EB8
:102CCC000A6E0F0E0B6EF3500A26F4500B220AC03C
:102CDC000CF00BC00DF00CC0D9FF0DC0DAFF09C011
:102CEC00DFFF12000001F1510001F25DD8A005D008
:102CFC00000E0001F26F000E18D00001F251010D10
:102D0C000201000EF324D96E0201020EF420DA6ED9
:102D1C00DF500001606F0001F22B0001606703D0EF
:102D2C00000E0001F26F0001605112000501085104
:102D3C00E7EC16F00001666F000166A104D0010EED
:102D4C0074EC15F003D0010E57EC15F0000166A3DE
:102D5C0004D0020E74EC15F003D0020E57EC15F0F3
:102D6C00000166A504D0030E74EC15F003D0030E1D
:102D7C0057EC15F01200000E0001656F000106D033
:102D8C000001665135EC17F00001652B000165510F
:102D9C00010D000161C063F0000162C064F0F350EA
:102DAC0000016327F4500001642363C0F6FF64C084
:102DBC00F7FF08000001F5CF66F000016667E0D769
:102DCC0012000001656F65C0EEF000016551D2EC98
:102DDC001BF00001656FFE0EF66E170EF76E090004
:102DEC00F5CF63F00900F5CF64F0030E0001635DCD
:102DFC00000E6459D8B009D04D2A030E4D6403D08F
:102E0C00000E4D6E02D00001659300016551120059
:102E1C00FE0EF66E170EF76E0900F5CF65F0090081
:102E2C00F5CF66F0030E0001655D000E6659D8A063
:102E3C000CD00F0E5A6E8B0E596E5AC058F059C0EA
:102E4C0057F0010E5B6E020E5C6E010E74EC15F009
:102E5C00020E74EC15F0030E74EC15F01200000168
:102E6C00606F800E0001F25DD8B010D00001F251FD
:102E7C00010D0201000EF324D96E0201020EF420A2
:102E8C00DA6E000160C0DFFF0001F22B800E000142
:102E9C00F25DD8B00DD00001F251010D0201000E0F
:102EAC00F324D96E0201020EF420DA6E000EDF6EEE
:102EBC001200000E0001676F000106D00001665180
:102ECC0035EC17F00001672B00016751010D000173
:102EDC0061C064F0000162C065F0F350000164272A
:102EEC00F4500001652364C0F6FF65C0F7FF0800CD
:102EFC000001F5CF66F0000163510001675DD8B0A9
:102F0C0003D000016667DAD712004650020AD8A433
:102F1C0003D085EC26F025D0000E466E3F661FD000
:102F2C0020EE01F03B50D9263C50DA22080EDF6E21
:102F3C0020EE02F03B50D9263C50DA22200EDE6EF9
:102F4C00040EDD6E3BC0D9FF3CC0DAFF0C0EDF6E09
:102F5C003BC0D9FF3CC0DAFF000EDB8E02D0000E66
:102F6C003F6E12000001616F1ED05B50FF0A000122
:102F7C00606F57C0D9FF58C0DAFF11D05C50FF0A00
:102F8C000001606F59C0D9FF5AC0DAFF08D05D50FC
:102F9C00FF0A0001606F94C1D9FF95C1DAFF0001EF
:102FAC006051DF160BD000016151010AD8B4DDD796
:102FBC00030AD8B4E3D7010AD8B4E9D71200000E3B
:102FCC00026E010E016EABEC12F00001F06F050EFB
:102FDC000001F06503D0000E0001F06F000E026ED0
:102FEC00050E016EABEC12F00001E56F060E000150
:102FFC00E56503D0040E0001E56F000E026E060EAF
:10300C00016EABEC12F00001EC6F030E0001EC65ED
:10301C0003D0000E0001EC6F1200000E0001616F76
:10302C00010E0001606FBDEC12F00001F06F050E97
:10303C000001F06503D0000E0001F06F000E0001DE
:10304C00616F050E0001606FBDEC12F00001E56FC1
:10305C00060E0001E56503D0040E0001E56F000EBD
:10306C000001616F060E0001606FBDEC12F00001F3
:10307C00EC6F030E0001EC6503D0000E0001EC6F49
:10308C001200000171C077F0000170C076F00001F1
:10309C006FC075F000016EC074F01DD0000176C0D9
:1030AC00F6FF000177C0F7FFF86A74C0D9FF75C04E
:1030BC00DAFF070EF76403D00800F55005D0F6CF01
:1030CC00E1FFF7CFE2FFE750DF6E0001764B772B85
:1030DC000001744B752B00017207D8A07307000117
:1030EC007229D8B47329D8B41200D8D70CD096EC66
:1030FC0012F031D09AEC12F02ED04BEC2BF02BD0EE
:10310C004AEC24F028D015C01BF016C01CF01C5043
:10311C00000AD8B404D07F0AD8B41BD01CD01B50E2
:10312C00010AD8B4EAD7030AD8B415D0010AD8B426
:10313C00E7D7060AD8B40FD0770AD8B40CD0010A56
:10314C00D8B409D0070AD8B4D5D7010AD8B4CFD788
:10315C0002D01B50FF0A12000600EACF2EF0E1CF7E
:10316C002FF0E2CF30F0D9CF31F0DACF32F0F3CF0D
:10317C0033F0F4CF34F0F6CF35F0F7CF36F0F8CF9C
:10318C0037F0F5CF38F055EC25F038C0F5FF37C0E7
:10319C00F8FF36C0F7FF35C0F6FF34C0F4FF33C07C
:1031AC00F3FF32C0DAFF31C0D9FF30C0E2FF2FC0CD
:1031BC00E1FF2EC0EAFF2DC0E9FF2CC0FBFF2BC0A6
:1031CC00FAFF1100000161C067F0000160C066F0F9
:1031DC0020D0000166C0F6FF000167C0F7FFF86A57
:1031EC00070EF76403D00800F55005D0F6CFE1FFC9
:1031FC00F7CFE2FFE75000016219D8A407D0000115
:10320C0067C061F0000166C060F013D00001664B2E
:10321C00672B00016407D8A0650700016429D8B4A6
:10322C006529D8A4D6D7000E0001616F000E0001ED
:10323C00606F120036D062C0D9FF63C0DAFFDF5076
:10324C000001666F60C0D9FF61C0DAFFDF5000017A
:10325C006619D8B420D062C0D9FF63C0DAFFDF5042
:10326C000001666F676B0001661F671F664B672B5B
:10327C0060C0D9FF61C0DAFFDF500001686F000148
:10328C006851000166250001606F000E0001672186
:10329C000001616F16D00001604B612B0001624B85
:1032AC00632B00016407D8A0650700016429D8B41A
:1032BC006529D8A4C0D7000E0001616F000E000173
:1032CC00606F1200000E4B6E000E426E000E406ED0
:1032DC00000E416E000E3F6E000E466ED9C0D9FF37
:1032EC00DAC0DAFF7F0EDF16040E0001D91BD9C03D
:1032FC00D9FFDAC0DAFF7F0EDF16040E0001D91BEE
:10330C003BC0D9FF3CC0DAFF7F0EDF16000E000178
:10331C00F86F000E0001FA6F000E0001F96F000E3D
:10332C000001D46F000E0001D66F000E0001D56FA6
:10333C00F4EC20F0000E166E030E156E000E186ED7
:10334C00000E176E000E1A6E000E196E7CEC18F043
:10335C006CEC21F01200FE0EF66E170EF76E0900E3
:10336C00F5CF60F00900F5CF61F0030E0001605D50
:10337C00000E6159D8A004D0010E4C6E070E5F6E82
:10338C00FE0EF66E170EF76E0900F5CF60F0090011
:10339C00F5CF61F0040E0001605D000E6159D8A0FC
:1033AC0002D0F30E5E6E4CC092FF000E966E010EB4
:1033BC000001636F8350FF0A5E140009D8A40CD07F
:1033CC008150FF0A0001606F3F0E00016017D8A406
:1033DC0003D0000E0001636F63C062F03F0E926E6B
:1033EC005FC096FF0001625112000001646F7D0EF8
:1033FC000001636F800E0001626F000E0001656FAB
:10340C0039D000016551010D000162C060F000016E
:10341C0063C061F0F35000016027F4500001612398
:10342C0060C0F6FF61C0F7FF0800F5500001641999
:10343C00D8A41ED00001EF51070D800E0001606F63
:10344C007D0E616FF35000016027F4500001612381
:10345C0000016551010DF35000016027F45000018B
:10346C00612360C0F6FF61C0F7FF0800F55008D07B
:10347C000001652B060E00016565C3D70001645180
:10348C00120002EE00F0800EEE6AE806FDE101EE9D
:10349C009EF0450EEE6AE806FDE100EED1F02B0E33
:1034AC00EE6AE806FDE100EE39F01E0EEE6AE80663
:1034BC00FDE1640EF66E360EF76E000EF86E01EE40
:1034CC0000F010EE9EF00900F5CFEEFFE550E15054
:1034DC00FAE11C0EF66E250EF76E000EF86E00EE7D
:1034EC00FCF010EE04F00900F5CFEEFFE550E150D2
:1034FC00FAE11C0EF66E180EF76E000EF86E00EE6A
:10350C0057F010EE09F00900F5CFEEFFE550E15051
:10351C00FAE1000EF86E0001EFEF15F0066E0401F3
:10352C00040E086E0401000E076E0150026E036A51
:10353C00D890023603360650046E056AD8900436CD
:10354C000536D89004360536025004260350052261
:10355C00D89004360536D890043605360450072624
:10356C000550082207C0D9FF08C0DAFFDF9E0166AC
:10357C0009D00650020D0001DD0EF324D96E0001B6
:10358C00000E08D00650020D0001D90EF324D96E9E
:10359C000001000EF420DA6E07C0DEFF08C0DDFF6C
:1035AC0007C0D9FF08C0DAFFDF9C20EE04F00750FB
:1035BC00D9260850DA22DF8C1200000E406E000E65
:1035CC00416E4650020AD8A41DD020EE01F03B50AB
:1035DC00D9263C50DA22080EDF6E20EE02F03B506A
:1035EC00D9263C50DA22280EDE6E040EDD6E3BC06E
:1035FC00D9FF3CC0DAFF480EDF6E3BC0D9FF3CC0A0
:10360C00DAFF27D00001F9510401265D0001FA51BF
:10361C0004012759D8B004D026C4F9F027C4FAF015
:10362C0080EC20F0000120EE02F00001D951D926E7
:10363C000001DA51DA22280EDE6E040EDD6ED9C0DE
:10364C00D9FFDAC0DAFF480EDF6ED9C0D9FFDAC075
:10365C00DAFF000EDB8E1200830F830F830F830FB4
:10366C00830F830F810F810F810F810F810F810FCA
:10367C00810F810F810F810F810F810F830F830FBA
:10368C00830F830F830F830F920F920F920F920F62
:10369C00920F920F960F960F960F960F960F920F02
:1036AC00920F920F920F920F10204080040820105E
:1036BC0002010408804020100804201008040102B4
:1036CC0001020408102080402010020100000E0EA0
:1036DC000E0E0E0E01020408102001020204081046
:1036EC002001020404020120100804028B0F0000C8
:1036FC000E0E0E0E0E0E0101010E026E0101A60E33
:10370C00016E000E046E0E0E036E000E066E1E0E83
:10371C00056EC7EC13F0000E026E020E016EABECE0
:10372C0012F00001F36F070E0001F36503D0000ED9
:10373C000001F36F000E026E040E016EABEC12F082
:10374C000001EF6F050E0001EF6503D0000E0001C4
:10375C00EF6F000E026E030E016EABEC12F0000167
:10376C00EA6F040E0001EA6503D0000E0001EA6F57
:10377C00000E026E080E016EABEC12F00001F46F3D
:10378C00010E0001F46503D0000E0001F46FE0ECB3
:10379C0012F0E5EC17F012000001626F0001F0511D
:1037AC00D8A437D04AD0E5C060F0010E0001616F9B
:1037BC000001602B03D00001D89061370001602F0D
:1037CC00FAD700016151FF0A00016217E5C060F0F1
:1037DC00EDC061F00001602B03D00001D89061377F
:1037EC000001602FFAD710D0E5C060F0FD0E00018B
:1037FC006027EDC061F00001602B03D00001D89070
:10380C0061370001602FFAD700016151000162138A
:10381C0014D00001E551000AD8B4C5D7010AD8B4B8
:10382C00C2D7030AD8B4BFD7010AD8B4DDD7070A68
:10383C00D8B4DAD7010AD8B4D7D700016251120034
:10384C000001706F000170C060F00001616B000E30
:10385C000001636F0C0E0001626F3EEC1DF0000165
:10386C0060510001716F0001EEA13FD0060E000106
:10387C0071653BD0070E0001715F000E0001636F94
:10388C000C0E0001626F000170C060F00001616BF2
:10389C000FEC20F0000160C068F0000161C069F01D
:1038AC00000E00016B6F050E00016A6FE7EC14F05F
:1038BC00530E00016E6F770E6F6F0001685100019F
:1038CC006E270001695100016F2300017151010D38
:1038DC00F35000016E27F45000016F236EC0F6FF09
:1038EC006FC0F7FF0800F55001D0000E1200010167
:1038FC00010E0001616F0101A60E0001606F000E48
:10390C000001636F0E0E0001626F000E0001656F07
:10391C001E0E0001646F1EEC15F0000E0001616FAD
:10392C00020E0001606FBDEC12F00001F36F070E88
:10393C000001F36503D0000E0001F36F000E0001CF
:10394C00616F040E0001606FBDEC12F00001EF6FAF
:10395C00050E0001EF6503D0000E0001EF6F000EA5
:10396C000001616F030E0001606FBDEC12F00001ED
:10397C00EA6F040E0001EA6503D0000E0001EA6F45
:10398C00000E0001616F080E0001606FBDEC12F0BB
:10399C000001F46F010E0001F46503D0000E00016C
:1039AC00F46F78EC13F013EC18F0120043665FD050
:1039BC00010E436E44665BD0010E446E4650020A03
:1039CC00D8A418D0000120EE01F00001D951D9265D
:1039DC000001DA51DA22000EDF6ED9C0D9FFDAC04D
:1039EC00DAFF480EDF6ED9C0D9FFDAC0DAFF000E5D
:1039FC00DB8E3DD04604D8A43AD0000E3F6E20EEAC
:103A0C0001F03950D9263A50DA22080EDF6E20EE3A
:103A1C0002F03950D9263A50DA22200EDE6E040E0E
:103A2C00DD6E39C0D9FF3AC0DAFF040EDF6E39C043
:103A3C00D9FF3AC0DAFF000EDB8E010E3F6E20EE8E
:103A4C0001F03B50D9263C50DA22080EDF6E20EEF6
:103A5C0002F03B50D9263C50DA22200EDE6E040ECA
:103A6C00DD6E3BC0D9FF3CC0DAFF800EDF6E12006A
:103A7C00000E0001656F00016151800AF36E800E2B
:103A8C00F35C000ED8B4605DD8B009D00001606D55
:103A9C000001611FD8B0612B010E0001656F0001A0
:103AAC006351800AF36E800EF35C000ED8B4625D35
:103ABC00D8B006D00001626D0001631FD8B0632B33
:103ACC00000163516211D8B426D0010E0001646F5D
:103ADC0006D00001D890623763370001642B0001D7
:103AEC0063AFF7D7000162510001605D00016351C3
:103AFC0000016159D8A008D0000162510001605F3B
:103B0C00000163510001615B0001D89063336233A3
:103B1C000001642FE7D700016551D8B406D000012D
:103B2C00606D0001611FD8B0612B60C060F061C096
:103B3C0061F01200000E0401286F000E0401296FC1
:103B4C0040D00001F88F0001E705D8A446D004014D
:103B5C00288343D00001F88F40D00001F88F040176
:103B6C0024BF0DD0040124510F0B016E0150020D26
:103B7C000001DD0EF324D96E0001000E0CD00401FF
:103B8C0024510F0B016E0150020D0001D90EF324CC
:103B9C00D96E0001000EF420DA6EDECF02F0DDCF1C
:103BAC0003F002C0D9FF03C0DAFFDFAE16D002C0AB
:103BBC00D9FF03C0DAFFDFA410D0010E0401286F77
:103BCC000CD0040120511F0B000AD8B4BAD7010A3B
:103BDC00D8B4C0D7030AD8B4C0D70001F8AF0DD001
:103BEC000401040E0001F66F0401280E0001F56FAC
:103BFC000001F881020E0001F96F1200056E0150F0
:103C0C00D8B409D00550020D0001D90EF324D96E99
:103C1C000001000E08D00550020D0001DD0EF3244A
:103C2C00D96E0001000EF420DA6EDECF06F0DDCF87
:103C3C0007F007500610D8A405D0000E026E000E37
:103C4C00016E40D020EE02F00650D9260750DA2241
:103C5C0002C0DEFF03C0DDFF20EE01F00650D926C6
:103C6C000750DA2204C0DFFF06C0D9FF07C0DAFF15
:103C7C00400EDF1606C0D9FF07C0DAFF000EDB8648
:103C8C0006C0D9FF07C0DAFF000EDB8E0150D8B496
:103C9C0009D00550020D0001D90EF324D96E000194
:103CAC00000E08D00550020D0001DD0EF324D96E74
:103CBC000001000EF420DA6E040EDF1A07C002F0C9
:103CCC0006C001F012000B6E59D0000EBD6E000E36
:103CDC00BA6E0F0EC16EFE0EF66E170EF76E090061
:103CEC00F5CF09F00900F5CF0AF0030E095C000EC0
:103CFC000A58D8A01DD0000EC26E0E0EC16E9E0EBC
:103D0C00C06EFE0EF66E170EF76E0900F5CF09F0B9
:103D1C000900F5CF0AF00950030A0A10D8A402D002
:103D2C00FE0E01D0F30E0001FE6F070E0001FF6FB7
:103D3C00000E896E3F0E926E000E8A6E9368F19E95
:103D4C00000E8B6E380E946E000E8C6EFEC095FFBE
:103D5C00848E000E8D6EFFC096FF81EC1BF018D088
:103D6C00130ED36E15D0600ED36E100E096E940E1A
:103D7C00E82EFED7092EFCD700D00AD00B50000A33
:103D8C00D8B4A3D7010AD8B4EBD7030AD8B4EBD76D
:103D9C001200D9C0D9FFDAC0DAFF000EDFBC010E69
:103DAC00026E040E0001D91B0001E951080AD8A4C7
:103DBC000CD0040122517F0B6E6E6E50D8B402D021
:103DCC00100E01D0040E0001E96F4604D8A42ED0C9
:103DDC00000120EE02F00001D951D9260001DA5180
:103DEC00DA22280EDE6E040EDD6E80EC20F04B50D5
:103DFC00020AD8A406D0D9C0D9FFDAC0DAFF040E63
:103E0C000DD0026606D0D9C0D9FFDAC0DAFF480E51
:103E1C0005D0D9C0D9FFDAC0DAFF080EDF6ED9C0E1
:103E2C00D9FFDAC0DAFF000EDB8E1BD00001D4AF55
:103E3C0016D00001D851D711D8B40FD0000120EE04
:103E4C00D7F001D80AD00500FA6EDE50FD6EDE50B8
:103E5C00FE6EF850FF6EFA5012000001D49F000E57
:103E6C00466E120000016A6F5CD0000EBD6E000E33
:103E7C00BA6E0F0EC16EFE0EF66E170EF76E0900BF
:103E8C00F5CF68F00900F5CF69F0030E0001685D0D
:103E9C00000E6959D8A01ED0000EC26E0E0EC16E57
:103EAC009E0EC06EFE0EF66E170EF76E0900F5CF65
:103EBC0068F00900F5CF69F000016851030A691137
:103ECC00D8A402D0FE0E01D0F30E0001FE6F070E37
:103EDC000001FF6F000E896E3F0E926E000E8A6E0F
:103EEC009368F19E000E8B6E380E946E000E8C6EE5
:103EFC00FEC095FF848E000E8D6EFFC096FF7DEC8C
:103F0C001CF01AD0130ED36E17D0600ED36E100E99
:103F1C000001686F940EE82EFED7682FFCD700D0F6
:103F2C000BD000016A51000AD8B49FD7010AD8B44B
:103F3C00E9D7030AD8B4E9D712002D0E456E54C048
:103F4C0027F0FD0E2716D8A45AD054C027F0D890CD
:103F5C0027323F0E27162750040D0401000EF324C0
:103F6C00396E0401040EF4203A6E3AC03CF039C0AC
:103F7C003BF0040E3B1A39C0D9FF3AC0DAFFDF30F0
:103F8C00E8320F0B0D0AD8A437D0000E296E24D0BE
:103F9C0020EE02F03950D9263A50DA22DECF27F043
:103FAC00DDCF28F027C0D9FF28C0DAFF2950010D3A
:103FBC000401200EF324E16E0401040EF420E26EE1
:103FCC00DFCFE7FF20EE02F03950D9263A50DA2243
:103FDC00DE2A000EDD22292A070E2964D9D720EE0D
:103FEC0002F03950D9263A50DA22200EDE6E040E39
:103FFC00DD6E68EC19F00CD08BEC17F009D054C0C6
:10400C0027F0FD0E27162750040AD8B4CFEC1EF06B
:10401C001200000E0001656F00016351800AF36EFF
:10402C00800EF35C000ED8B4625DD8B009D00001EC
:10403C00626D0001631FD8B0632B010E0001656F28
:10404C0000016151800AF36E800EF35C000ED8B44F
:10405C00605DD8B009D00001606D0001611FD8B05F
:10406C00612B010E0001651B000E0001676F000E35
:10407C000001666F000163516211D8B42CD0010E9F
:10408C000001646F06D00001D890623763370001DD
:10409C00642B000163AFF7D70001D8906637673700
:1040AC00000162510001605D000163510001615922
:1040BC00D8A00AD0000162510001605F0001635179
:1040CC000001615B000166810001D89063336233AB
:1040DC000001642FE1D700016551D8B406D000016E
:1040EC00666D0001671FD8B0672B66C060F067C0B3
:1040FC0061F01200080E016E080E0001F95D000E51
:10410C000001FA59D8B00BD0F9C001F04B6602D0BF
:10411C00010E04D04B04D8A402D0020E4B6E0150F9
:10412C000001F95F000E0001FA5B000120EE01F0C6
:10413C000001D951D9260001DA51DA2201C0DFFF82
:10414C000401040E0101A36F0401280E0101A26FEA
:10415C000001F8A11FD03FD00001F5C0F6FF00010F
:10416C00F6C0F7FFF86AA2C1D9FFA3C1DAFF070EA8
:10417C00F76403D00800F55005D0F6CFE1FFF7CF78
:10418C00E2FFE750DF6E0001F54BF62B0101A24B6D
:10419C00A32B01060166E0D720D00001F5C0F6FF85
:1041AC000001F6C0F7FFF86AA2C1D9FFA3C1DAFF7C
:1041BC00070EF76403D00800F55005D0F6CFE1FFE9
:1041CC00F7CFE2FFE750DF6E0001F54BF62B010154
:1041DC00A24BA32B01060166E0D712000401203983
:1041EC00E832030B0009D8A470D04ED00001F88F30
:1041FC00080E0001E96F69D0BCEC27F066D0E4EC46
:10420C0021F063D0000E0001F66F520E0001F56F25
:10421C0015D0A0EC1DF059D053EC2CF056D0040165
:10422C002451010D530E256E000E266EF3502526DB
:10423C00F450262225C0F5F026C0F6F00001F881D6
:10424C00010E0001F96F0001F88F3FD00001F88FCB
:10425C0004012451010D530EF324D96E000EF420E9
:10426C00DA6E040122C4DFFF30D0000E166E020E8F
:10427C00156E000E186E000E176E000E1A6E000EE4
:10428C00196E7CEC18F021D004012151000AD8B42D
:10429C00C0D7010AD8B4C0D7020AD8B4BDD7060A11
:1042AC00D8B4A4D7030AD8B4A7D7010AD8B4DDD799
:1042BC000F0AD8B4A7D7010AD8B4A1D7030AD8B427
:1042CC00AED7010AD8B4C2D7070A12006D98000104
:1042DC00F8BF39D00001D4AF0BD0020E466E416648
:1042EC0002D0E3EC1AF0000E446E000E436E65D063
:1042FC0020EE01F03B50D9263C50DA22080EDF6E3E
:10430C0020EE02F03B50D9263C50DA22200EDE6E15
:10431C00040EDD6E3BC0D9FF3CC0DAFF0C0EDF6E25
:10432C003BC0D9FF3CC0DAFF000EDB8ED9C0D9FFF1
:10433C00DAC0DAFF040EDF6ED9C0D9FFDAC0DAFFBB
:10434C00000EDB8E3AD0040120AF0FD0010E466E6A
:10435C00406602D0E3EC1AF0000E446E000E436E81
:10436C0042662BD0DCEC1CF028D0020E466E20EE00
:10437C0001F03B50D9263C50DA22080EDF6E20EEBD
:10438C0002F03B50D9263C50DA22200EDE6E040E91
:10439C00DD6E3BC0D9FF3CC0DAFF040EDF6E3BC0C4
:1043AC00D9FF3CC0DAFF000EDB8E000E446E000E0F
:1043BC00436E426602D0DCEC1CF012000001F88F58
:1043CC000F0E026E710E016E000E046E000E036E67
:1043DC00000E066E010E056EC7EC13F00401040E00
:1043EC00026E0401000E016E000E046E000E036ED0
:1043FC00000E066E200E056EC7EC13F06D8C000ED1
:10440C001D6E19D01D50010D0001E10EF324D96E63
:10441C000001000EF420DA6E000EDF6E1D50010D4F
:10442C000001E30EF324D96E0001000EF420DA6EC5
:10443C00000EDF6E1D2A010E1D64E4D7000E026E05
:10444C00530E016E000E046E000E036E000E066E0F
:10445C00010E056EC7EC13F06D9C0401040E0001F7
:10446C00DA6F0401080E0001D96F0401040E3A6ED4
:10447C000401000E396E3AC03CF039C03BF022C446
:10448C0052F0526602D0100E0FD0000E166E010EB6
:10449C00156E000E186E520E176E000E1A6E010E6F
:1044AC00196E7CEC18F0200E0001E96F1200000E62
:1044BC000001696F000E00016A6F000E00016C6F45
:1044CC0012D000016C51010D0101D80EF324D96EEC
:1044DC000101010EF420DA6E010EDF6402D000013E
:1044EC00692B00016C2B070E00016C65EAD7000EDE
:1044FC0000016C6F12D000016C51010D0101C40E52
:10450C00F324D96E0101010EF420DA6E010EDF6482
:10451C0002D000016A2B00016C2B0B0E00016C65A4
:10452C00EAD7000E00016B6F010E0001696507D020
:10453C00010E00016A6503D0010E00016B6F6BC0A8
:10454C0068F00101010E0001616F0101D80E00013C
:10455C00606F000E0001636F000E0001626F000EB1
:10456C000001656F080E0001646F1EEC15F001016F
:10457C00010E0001616F0101C40E0001606F000E9D
:10458C000001636F000E0001626F000E0001656F89
:10459C000C0E0001646F1EEC15F000016851120046
:1045AC00000163C06BF0000162C06AF0000161C0E1
:1045BC0069F0000160C068F00001685100016A5D9B
:1045CC000001695100016B59D8B044D000016AC098
:1045DC0066F000016BC067F00001645100016627B2
:1045EC000001655100016723000166510001685DFF
:1045FC000001675100016959D8B02CD000016451F9
:10460C0000016A270001655100016B230001645110
:10461C0000016827000165510001692300016A0748
:10462C00D8A06B076AC0D9FF6BC0DAFF000168071E
:10463C00D8A0690768C0E1FF69C0E2FFDFCFE7FFE0
:10464C0000016407D8A06507000165516411D8B456
:10465C001FD0E4D7000165516411D8B419D06AC0D9
:10466C00D9FF6BC0DAFF68C0E1FF69C0E2FFDFCFA2
:10467C00E7FF00016A4B6B2B0001684B692B0001B3
:10468C006407D8A06507000165516411D8A4E7D769
:10469C0012000001646F00016051D8B40AD000010F
:1046AC006451020D0001D90EF324D96E0001000EE5
:1046BC0009D000016451020D0001DD0EF324D96E06
:1046CC000001000EF420DA6E0001DECF65F000016F
:1046DC00DDCF66F0000166516511D8A407D0000E3D
:1046EC000001616F000E0001606F4ED0000120EEE2
:1046FC0002F000016551D92600016651DA22000151
:10470C0061C0DEFF000162C0DDFF000120EE01F0A0
:10471C0000016551D92600016651DA22000163C0FF
:10472C00DFFF65C0D9FF66C0DAFF400EDF1665C03B
:10473C00D9FF66C0DAFF000EDB8665C0D9FF66C004
:10474C00DAFF000EDB8E00016051D8B40AD00001F4
:10475C006451020D0001D90EF324D96E0001000E34
:10476C0009D000016451020D0001DD0EF324D96E55
:10477C000001000EF420DA6E040EDF1A000166C090
:10478C0061F0000165C060F012000001726F000161
:10479C00F351040AD8B405D00001F351050AD8A48A
:1047AC0023D04F0E000172651FD0540E0001725DB4
:1047BC00D8B01AD0B00E000172250001686F00014C
:1047CC00696BFF0E6923000E00016B6F030E000175
:1047DC006A6FE7EC14F0C00E0001682500016E6FE3
:1047EC007F0E000169214DD0000E0001636F0C0E8D
:1047FC000001626F000172C060F00001616B0FEC90
:10480C0020F0000160C068F0000161C069F0000E8A
:10481C0000016B6F240E00016A6FE7EC14F08E0E32
:10482C000001706F770E716F0001685100017027E5
:10483C000001695100017123000E0001636F0C0E21
:10484C000001626F000172C060F00001616B3EEC10
:10485C001DF0000160C068F0000161C069F0000E3D
:10486C0000016B6F030E00016A6FE7EC14F000019E
:10487C0068510001702500016E6F00016951000143
:10488C00712100016F6F1200040120511F0B016E8A
:10489C000104D8A47BD004012451D8A477D00401FE
:1048AC002151060AD8B41FD027D05204D8A424D042
:1048BC007D0E0001F66FE60E0001F56F000E000193
:1048CC00FA6F090E0AD07C0E0001F66FE00E0001A3
:1048DC00F56F000E0001FA6F400E0001F96FC00E6B
:1048EC000001F86F09D004012351210AD8B4DDD797
:1048FC00030AD8B4E8D7010A04012039E832030BC3
:10490C00016E0104D8A442D02DD0DDEC13F03ED0C2
:10491C00000E0001F66F560E0001F56F000E00013F
:10492C00FA6F010E0001F96FC10E13D0800E000159
:10493C00F86F23C456F02AD0000E0001F66F550E06
:10494C000001F56F000E0001FA6F010E0001F96F06
:10495C00810E0001F86F1AD0800E0001F86F22C48E
:10496C0055F014D004012151010AD8B40FD0030A18
:10497C00D8B4CED7010AD8B4DFD70A0AD8B4C5D771
:10498C00030AD8B4D3D7010AD8B4E6D71200000171
:10499C00746F0001745126EC1CF00001756F00015E
:1049AC0074C060F00001616B000E0001636F0C0EAF
:1049BC000001626F0FEC20F0000160510001766F76
:1049CC00000174C060F00001616B000E0001636FA8
:1049DC000C0E0001626F3EEC1DF0000160510001F5
:1049EC00776F00017551D8B443D00001755156D082
:1049FC00000176510C0DD30E0001726F750E1FD095
:104A0C00000176510C0D730E0001726F750E17D0EC
:104A1C00000176510C0D330E0001726F760E0FD023
:104A2C00000176510C0D930E0001726F760E07D0BB
:104A3C00000176510C0DF30E0001726F760E736F40
:104A4C00F35000017227F4500001732300017751D9
:104A5C00010DF35000017227F4500001732372C052
:104A6C00F6FF73C0F7FF08000001F5CF75F012D008
:104A7C000001E651000AD8B4DBD7010AD8B4B8D784
:104A8C00030AD8B4BDD7010AD8B4C2D7070AD8B420
:104A9C00C7D7CED700017551FBEC19F012000001FD
:104AAC00E905D8B46DBA07D0000E686E69806988C4
:104ABC00020E0001E96F68B469A403D0689402EC9B
:104ACC0015F06DB282D068B069A007D0FCEC28F06C
:104ADC00A08A040E0001E96F689068B869A803D039
:104AEC009DEC13F0689868AC18D069AC0ED0000E31
:104AFC00166E730E156E000E186E000E176E000EED
:104B0C001A6E010E196E7CEC18F0689C4550D8A4F6
:104B1C004506456602D0DCEC1CF068BA69AA02D0E6
:104B2C0091EC15F068B269A20FD07F0E166E156865
:104B3C00000E186E000E176E000E1A6E010E196E16
:104B4C007CEC18F0000E6A6E040E0001E95DD8B022
:104B5C0069A63BD0000E2A6E35D068A636D06CCF35
:104B6C0054F05430E832E8320F0B486E689654B467
:104B7C0009D04850010D0001E30EF324D96E000159
:104B8C00000E08D04850010D0001E10EF324D96E3F
:104B9C000001000EF420DA6E0001DF70486603D0CD
:104BAC00A3EC1FF00ED0000E166E720E156E000EDA
:104BBC00186E540E176E000E1A6E000E196E7CECE9
:104BCC0018F02A2A030E2A64C8D7A19A12007F0E65
:104BDC000001626F720E0001616FC1EC16F0FE0EE7
:104BEC00F66E170EF76E09000001F5CF60F00A00A3
:104BFC000001F5CF61F0CDEC14F035EC17F0280E78
:104C0C0035EC17F07F0E0001626FD40E0001616F5E
:104C1C00C1EC16F0000E0001616F000E0001606F18
:104C2C00CDEC14F035EC17F0370E35EC17F0000E18
:104C3C000001616F010E0001606FCDEC14F035ECDA
:104C4C0017F0000E0001616F040E0001606FCDECD7
:104C5C0014F035EC17F0280E35EC17F07E0E000131
:104C6C00626F250E0001616FC1EC16F056EC13F06B
:104C7C007F0E0001626FDE0E0001616FC1EC16F059
:104C8C00F0EC12F07F0E0001626FE20E0001616F1A
:104C9C00C1EC16F023EC13F07F0E0001626FE60EF0
:104CAC000001616FC1EC16F001EC13F07F0E0001F6
:104CBC00626FEA0E0001616FC1EC16F045EC13F067
:104CCC007F0E0001626FEE0E0001616FC1EC16F0F9
:104CDC0012EC13F07F0E0001626FF20E0001616F97
:104CEC00C1EC16F034EC13F07F0E0001626FDA0E9B
:104CFC000001616FC1EC16F067EC13F0120020EEAE
:104D0C0001F03950D9263A50DA22DF50026E0250A7
:104D1C000001D55D000E0001D659D8A0D5C002F017
:104D2C0002500001D55F000E0001D65B000E016E33
:104D3C0014D00150010D0401280EF324D96E040186
:104D4C00040EF420DA6ED1C0E1FFD2C0E2FFDFCF57
:104D5C00E7FF0001D14BD22B012A0250015CD8A0F5
:104D6C00E8D70001D651D511D8B42BD020EE01F0E4
:104D7C003B50D9263C50DA22080EDF6E20EE02F0B2
:104D8C003B50D9263C50DA22280EDE6E040EDD6E26
:104D9C0039C0D9FF3AC0DAFFDFBC06D03BC0D9FF1F
:104DAC003CC0DAFF480E05D03BC0D9FF3CC0DAFF4F
:104DBC00080EDF6E3BC0D9FF3CC0DAFF000EDB8E65
:104DCC0038D020EE01F03B50D9263C50DA22080EA8
:104DDC00DF6E20EE02F03B50D9263C50DA22200E3A
:104DEC00DE6E040EDD6E3BC0D9FF3CC0DAFF040E54
:104DFC00DF6E3BC0D9FF3CC0DAFF000EDB8E00013A
:104E0C00D851D711D8B40FD0000120EED7F001D86B
:104E1C000AD00500FA6EDE50FD6EDE50FE6EF850C4
:104E2C00FF6EFA5012000001D49F426602D0DCECF7
:104E3C001CF0120000017C6FFE0EF66E170EF76E62
:104E4C000900F5CF79F00900F5CF7AF0020E0001D8
:104E5C00795D000E7A59D8A020D000017C510C0D40
:104E6C00130E0001796F750E7A6FF35000017927DC
:104E7C00F45000017A2300017851010DF350000128
:104E8C007927F45000017A2379C0F6FF7AC0F7FF36
:104E9C0008000001F5CF7BF008D000017C510C0D0F
:104EAC00F3500001782500017B6F00017851010D52
:104EBC000101C40EF324D96E0101010EF420DA6E47
:104ECC00DF2A00017C51010D0101D80EF324D96EAB
:104EDC000101010EF420DA6EDF2A00017B51CDECCA
:104EEC0024F000017D6FDF0E00017D651BD0E80E04
:104EFC0000017D5DD8B016D07DC079F0200E000188
:104F0C007927010E00017A6F0001792B03D0000183
:104F1C00D8907A370001792FFAD700017A51000125
:104F2C00FB1323D000017D51F00AD8A403D001015A
:104F3C00D1811BD00001FD51800A0001796F080E50
:104F4C00800A0001795DD8B010D00001FD51010D2F
:104F5C000101D00EF324D96E0101010EF420DA6E9A
:104F6C0000017BC0DFFF0001FD2B1200040120516A
:104F7C00800AD8A499D0C00E0001F86F89D07F0E9A
:104F8C000001F66FAE0E0001F56F000E0001FA6F16
:104F9C00120E0001F96F88D00401226775D004014C
:104FAC002251020D8C0EF324F66E770EF420F76E60
:104FBC0009000001F5CFF5F00A000001F5CFF6F07D
:104FCC00020E0001F525016E000E0001F621026EA5
:104FDC0001C0F6FF02C0F7FFF86A070EF76403D0B2
:104FEC000800F55005D0F6CFE1FFF7CFE2FFE75010
:104FFC000001F96F030E0001F525016E000E000192
:10500C00F621026E01C0F6FF02C0F7FFF86A070E28
:10501C00F76403D00800F55005D0F6CFE1FFF7CFC9
:10502C00E2FFE7500001FA6F3FD0030E0401225D4E
:10503C00D8B02AD004012251020D820EF324F66E50
:10504C00770EF420F76E09000001F5CFF5F00A0099
:10505C000001F5CFF6F00001F5C0F6FF0001F6C037
:10506C00F7FFF86A070EF76403D00800F55005D077
:10507C00F6CFE1FFF7CFE2FFE750016E01500001E0
:10508C00F96F0001FA6B10D0000E0001F86F0CD014
:10509C0004012351010AD8B472D7030AD8B47CD7BF
:1050AC00010AD8B4C2D7F0D71200020E0001816FEA
:1050BC0078C0D9FF79C0DAFFDF5000017F6F020E94
:1050CC000001826F86D000018251010DF350000166
:1050DC007825D96EF45000017921DA6EDF50000189
:1050EC00806F0001805126EC1CF00001836F0001E1
:1050FC00836706D000018051CDEC24F00001836F52
:10510C0000018351D8B463D0080E0001815DD8B082
:10511C005ED000018351900AD8A402D0010E06D0B3
:10512C0000018351910AD8A404D0000E0001ED6F48
:10513C003ED000018351390AD8A425D0020E0001BB
:10514C007A250001606F000E00017B210001616F68
:10515C00000183C062F00001636B000E0001656FFB
:10516C00060E0001646FE8EC18F0000161510001BB
:10517C006011D8A41CD08AEC13F00009D8B417D055
:10518C00010E471A14D000018351270AD8A40FD05E
:10519C007FC07EF0220E00017E17D8B408D08AECB6
:1051AC0013F00009D8B403D0870E0001836F0001FF
:1051BC008151010DF35000017C25D96EF450000192
:1051CC007D21DA6E000183C0DFFF0001812B00011D
:1051DC00822B070E0001826576D77CC0D9FF7DC07B
:1051EC00DAFF00017FC0DFFF010E1200A09A000E53
:1051FC006A6E000E686E000E706E0F0E026E710EEF
:10520C00016E000E046E000E036E000E066E010E93
:10521C00056EC7EC13F0160E6F6E9F0E6B6E7B0E49
:10522C00696E000E096E0FD00950040D0401000EBA
:10523C00F324D96E0401040EF420DA6EDE6ADE6A01
:10524C00DE6ADD6A092A070E0964EED76D8C000E42
:10525C006E6E6D986D9C0DD06896000E0001F86F07
:10526C00000E0001D46F000E0001D66F000E00017D
:10527C00D56F68B6F1D7010E436E010E446E000E69
:10528C00406E000E416E000E0001E86F000E096EBC
:10529C0035D00950020D0001D90EF324D96E00014E
:1052AC00000EF420DA6E000EDE6E000EDD6E09507C
:1052BC00020D0001DD0EF324D96E0001000EF42066
:1052CC00DA6E000EDE6E000EDD6E0950010D00016F
:1052DC00E10EF324D96E0001000EF420DA6E000EFC
:1052EC00DF6E0950010D0001E30EF324D96E0001AD
:1052FC00000EF420DA6E000EDF6E092A010E09642E
:10530C00C8D70401040E0001DA6F0401080E000175
:10531C00D96F160E706E040E0401036F200E04017B
:10532C00026F080E0401016F040E0401006F0401EA
:10533C00008F000E526E000E0001E96F1200A09A51
:10534C00000E6A6E000E686E000E706E0F0E00017D
:10535C00616F710E0001606F000E0001636F000E33
:10536C000001626F000E0001656F010E0001646F99
:10537C001EEC15F0160E6F6E9F0E6B6E7B0E696E2B
:10538C00000E0001686F11D000016851040D04017A
:10539C00000EF324D96E0401040EF420DA6EDE6ADA
:1053AC00DE6ADE6ADD6A0001682B070E00016865A3
:1053BC00EBD76D8C000E6E6E6D986D9C0DD0689653
:1053CC00000E0001F86F000E0001D46F000E0001FA
:1053DC00D66F000E0001D56F68B6F1D7010E436E83
:1053EC00010E446E000E406E000E416E000E000168
:1053FC00E86F000E0001686F3AD000016851020D91
:10540C000001D90EF324D96E0001000EF420DA6EDF
:10541C00000EDE6E000EDD6E00016851020D000103
:10542C00DD0EF324D96E0001000EF420DA6E000EAE
:10543C00DE6E000EDD6E00016851010D0001E10E03
:10544C00F324D96E0001000EF420DA6E000EDF6E2C
:10545C0000016851010D0001E30EF324D96E000127
:10546C00000EF420DA6E000EDF6E0001682B010EC8
:10547C0000016865C2D70401040E0001DA6F040153
:10548C00080E0001D96F160E706E040E0401036F26
:10549C00200E0401026F080E0401016F040E0401BA
:1054AC00006F0401008F000E526E000E0001E96FB8
:1054BC001200D8D00001A7C084F00001A6C083F070
:1054CC000001A9C086F00001A8C085F00001ABC0A6
:1054DC0088F00001AAC087F07A0E00018A6FFA0EDC
:1054EC000001896F7B0E00018C6F4E0E00018B6FDB
:1054FC007B0E00018E6FA20E00018D6F10EC37F049
:10550C00C3D00001A7C084F00001A6C083F0000145
:10551C00A9C086F00001A8C085F00001ABC088F0DE
:10552C000001AAC087F0790E00018A6F560E0001A7
:10553C00896F790E00018C6FAA0E00018B6F790EAA
:10554C0000018E6FFE0E00018D6F10EC37F09CD0B9
:10555C000001A7C084F00001A6C083F00001A9C01F
:10556C0086F00001A8C085F00001ABC088F00001F6
:10557C00AAC087F0780E00018A6FAE0E0001896F09
:10558C00790E00018C6F020E00018B6F790E0001F9
:10559C008E6F020E00018D6F10EC37F075D000018C
:1055AC00A7C084F00001A6C083F00001A9C086F05A
:1055BC000001A8C085F00001ABC088F00001AAC0B2
:1055CC0087F07A0E00018A6F520E0001896F7A0EF5
:1055DC0000018C6FA60E00018B6F7A0E00018E6F8E
:1055EC00A60E00018D6F10EC37F04ED00001A7C055
:1055FC0084F00001A6C083F00001A9C086F0000170
:10560C00A8C085F00001ABC088F00001AAC087F0EB
:10561C007B0E00018A6FF60E0001896F7C0E000173
:10562C008C6F4A0E00018B6F7C0E00018E6F4A0E40
:10563C0000018D6F10EC37F027D00001A7C079F076
:10564C000001A6C078F00001A9C07BF00001A8C041
:10565C007AF00001ABC07DF00001AAC07CF05BECDD
:10566C0028F012D00001F051010AD8B44AD7030A2D
:10567C00D8B46ED7010AD8B41DD7070AD8B48FD7BF
:10568C00010AD8B4B3D7D9D71200000E01019F6F0D
:10569C00000E01019E6F000E0501086F1E0E096EB3
:1056AC00010E54EC16F0000E016E0501050E036E92
:1056BC000501080E026E010E046E010E04EC1EF0C4
:1056CC0001C0A0F102C0A1F1FE0EF66E170EF76E2E
:1056DC000900F5CF0FF00900F5CF10F00F50030AB9
:1056EC001010D8A440D00F0E01013B6F960E010193
:1056FC003A6F000E116E17D01150010D0101840E7E
:10570C00F324D96E0101010EF420DA6E1150010D53
:10571C0001017C0EF324E16E0101010EF420E26E16
:10572C00DFCFE7FF112A070E1164E6D7000E126EC9
:10573C0017D01250010D01015C0EF324D96E01013A
:10574C00010EF420DA6E1250010D0101500EF324FB
:10575C00E16E0101010EF420E26EDFCFE7FF122AA9
:10576C000B0E1264E6D7FE0EF66E170EF76E0900DE
:10577C00F5CF0FF00900F5CF10F0040E0F5C000E02
:10578C001058D8A080D0000E136E2FD01350020DDD
:10579C000101400EF324D96E0101010EF420DA6EE2
:1057AC001350020D0101300EF324E16E0101010EC4
:1057BC00F420E26EDECFE6FFDDCFE5FF1350010DE6
:1057CC0001018C0EF324D96E0101010EF420DA6E66
:1057DC001350010D01017C0EF324E16E0101010E49
:1057EC00F420E26EDFCFE7FF132A070E1364CED747
:1057FC00000E146E2FD01450020D0101180EF3245C
:10580C00D96E0101010EF420DA6E1450020D010163
:10581C00000EF324E16E0101010EF420E26EDECFE6
:10582C00E6FFDDCFE5FF1450010D0101680EF324F6
:10583C00D96E0101010EF420DA6E1450010D010134
:10584C00500EF324E16E0101010EF420E26EDFCF65
:10585C00E7FF142A0B0E1464CED7FE0EF66E170E4D
:10586C00F76E0900F5CF0FF00900F5CF10F0050E1B
:10587C000F5C000E1058D8A006D0010E01015A6F13
:10588C00020E01015B6F170ED0EC12F0A2EC12F0BD
:10589C0001C0A4F102C0A5F1120004012205D8A494
:1058AC0012D0040120511F0B0009D8A40CD0000108
:1058BC00F88F04012151030AD8A402D0010E01D0A3
:1058CC00000E0001E76F0401226744D1040120514E
:1058DC001F0B020AD8A43ED1040124510F0B00095E
:1058EC00D8B438D1040124510F0B1D6E020E1D5C6F
:1058FC00D8B030D10001E951200AD8A42BD1000135
:10590C00F88F040124BF1FD0040124510F0B1D6E0E
:10591C001D50020D0001DD0EF324D96E0001000EA6
:10592C00F420DA6EDECF23F0DDCF24F00401245115
:10593C000F0B1D6E1D50010D0001E30EF324D96EEB
:10594C000001000E1ED0040124510F0B1D6E1D50C2
:10595C00020D0001D90EF324D96E0001000EF420C3
:10596C00DA6EDECF23F0DDCF24F0040124510F0BCF
:10597C001D6E1D50010D0001E10EF324D96E0001C6
:10598C00000EF420DA6EDF50226E22B002D0239487
:10599C0001D02384040124BF0DD0040124510F0B2A
:1059AC001D6E1D50020D0001DD0EF324D96E000199
:1059BC00000E0CD0040124510F0B1D6E1D50020D56
:1059CC000001D90EF324D96E0001000EF420DA6E1A
:1059DC0023C0DEFF24C0DDFF04012151030AD8A43B
:1059EC0033D023C0D9FF24C0DAFFDFAE20D00401AE
:1059FC0024BF0DD0040124510F0B1D6E1D50010D41
:105A0C000001E30EF324D96E0001000E0CD004014A
:105A1C0024510F0B1D6E1D50010D0001E10EF324DE
:105A2C00D96E0001000EF420DA6E0001DF8223C073
:105A3C00D9FF24C0DAFF000EDB8423C0D9FF24C0B9
:105A4C00DAFF000EDB8E86D0040E231A23C0D9FF9A
:105A5C0024C0DAFFDFAE1BD023C0D9FF24C0DAFF8D
:105A6C007F0EDF1623C0D9FF24C0DAFF000EDB8CBB
:105A7C00000E166E050E156E24C018F023C017F01C
:105A8C00000E1A6E020E196E7CEC18F006D023C0B4
:105A9C00D9FF24C0DAFF000EDB8C040E231A22B2CD
:105AAC0006D023C0D9FF24C0DAFFDFAE35D0040105
:105ABC0024BF0DD0040124510F0B1D6E1D50010D80
:105ACC000001E30EF324D96E0001000E0CD004018A
:105ADC0024510F0B1D6E1D50010D0001E10EF3241E
:105AEC00D96E0001000EF420DA6E0001DF9223C0A3
:105AFC00D9FF24C0DAFF3B0EDF16000E166E050E22
:105B0C00156E24C018F023C017F0000E1A6E020E8A
:105B1C00196E7CEC18F006D023C0D9FF24C0DAFF34
:105B2C003B0EDF16040124510F0B1D6E1D50010D91
:105B3C00700E1E6E0F0E1F6EF3501E26F4501F2299
:105B4C001EC020F01FC021F020C0D9FF21C0DAFFF9
:105B5C00FE0EDF161200020E0001726FC7D100019B
:105B6C007251010DF35000016C25D96EF4500001F7
:105B7C006D21DA6E680E0CD000017251010DF350DC
:105B8C0000016C25D96EF45000016D21DA6E690E9E
:105B9C00DF6EAAD100017251010DF35000016C258A
:105BAC00D96EF45000016D21DA6EDF508A0AD8B438
:105BBC00B9D0010AD8B4B6D01B0AD8B4D0D7010AD0
:105BCC00D8B4DAD791D10001EF51020AD8B405D07C
:105BDC000001EF51050AD8A487D16CC0D9FF6DC064
:105BEC00DAFF000EDB8400017251010DF35000014D
:105BFC006C250001606FF45000016D210001616F94
:105C0C0000017251010D00016CC06EF000016DC0FD
:105C1C006FF0F35000016E27F45000016F23010E5A
:105C2C0000016E27000E6F236EC062F06FC063F030
:105C3C00000172510001706F716B0001701F711FB8
:105C4C00704B712B070E000170250001646F000E64
:105C5C00000171210001656FD6EC22F0000120EEED
:105C6C0007F000016C51D92600016D51DA22000EAB
:105C7C00DF6E0001720738D100017251010DF35033
:105C8C0000016C25D96EF45000016D21DA6EDF50E5
:105C9C00650AD8B498D7EF0AD8B444D0010AD8B45E
:105CAC0041D022D100017251010DF35000016C253D
:105CBC00D96EF45000016D21DA6E2C0E72D00001F9
:105CCC007251010DF35000016C25D96EF450000196
:105CDC006D21DA6E2A0E65D000017251010DF35060
:105CEC0000016C25D96EF45000016D21DA6EDF5085
:105CFC008A0AD8B417D0010AD8B414D01B0AD8B465
:105D0C00D1D7010AD8B4DBD7EFD000017251010D05
:105D1C00F35000016C25D96EF45000016D21DA6E40
:105D2C00350E86D000017251010DF35000016C2527
:105D3C00D96EF45000016D21DA6E2C0E29D70001BA
:105D4C007251010DF35000016C25D96EF450000115
:105D5C006D21DA6EDF508A0AD8B4E4D7010AD8B4C0
:105D6C00E1D71B0AD8B4D1D7010AD8B4CED7BCD04E
:105D7C0000017251010DF35000016C25D96EF450E5
:105D8C0000016D21DA6E8A0E0CD000017251010DEA
:105D9C00F35000016C25D96EF45000016D21DA6EC0
:105DAC008B0EDF6E6CC0D9FF6DC0DAFF030EDF12F5
:105DBC009BD000017251010DF35000016C25D96E7E
:105DCC00F45000016D21DA6EDF50900AD8B4D0D7B0
:105DDC00010AD8B4DAD788D000017251010DF35002
:105DEC0000016C25D96EF45000016D21DA6E350E70
:105DFC00CFD600017251010DF35000016C25D96E04
:105E0C00F45000016D21DA6EDF50900AD8B4E4D75B
:105E1C00010AD8B4E1D768D000017251010DF350DA
:105E2C0000016C25D96EF45000016D21DA6E2C0E38
:105E3C00DF6E6CC0D9FF6DC0DAFF000EDB8454D06E
:105E4C0000017251010DF35000016C25D96EF45014
:105E5C0000016D21DA6EDF50900AD8B4DDD7010A4B
:105E6C00D8B4DAD741D000017251010DF3500001C2
:105E7C006C25D96EF45000016D21DA6E2C0EDF6E9C
:105E8C006CC0D9FF6DC0DAFF000EDB822DD0000193
:105E9C007251010DF35000016C25D96EF4500001C4
:105EAC006D21DA6EDF50900AD8B4DDD7010AD8B470
:105EBC00DAD71AD00001F351000AD8B46BD6010A14
:105ECC00D8B4DAD6030AD8B407D7010AD8B437D76E
:105EDC00070AD8B46ED7010AD8B48BD7030AD8B442
:105EEC00AFD7010AD8B4D3D70001722B070E00012B
:105EFC007265E0D71200000E0001C26F5DEC22F05B
:105F0C000009D8B410D083D10001FD51010D01015D
:105F1C00D00EF324D96E0101010EF420DA6E0E0EB0
:105F2C00DF6E0001FD2B0001FD51800A780FD8A017
:105F3C00EBD70001EB51060D0101A60EF324000175
:105F4C00606F0101010EF4200001616F0101010E6F
:105F5C000001636F0101D20E0001626F000E00019F
:105F6C00656F060E0001646FD6EC22F0FBC0D0F119
:105F7C000001F451D8B403D04E500101D01396C196
:105F8C00C0F0220E0001C017D8A40BD0FBC0C0F08B
:105F9C00220E0001C017D8B404D00001FB51220B13
:105FAC004E6E0001EA5100080001EB25050F0001BF
:105FBC00C46F040E0001C46503D0050E0001C45F5C
:105FCC000001C451040F0001C66F040E0001C66528
:105FDC0003D0050E0001C65F020E0001FD6F000E1E
:105FEC000001C56F53D00001C451060DA60E00016F
:105FFC00C06F010EC16FF3500001C027F4500001B7
:10600C00C1230001C551010DF3500001C025D96E0B
:10601C00F4500001C121DA6EDF500001C36F0001A2
:10602C00C651060DA60E0001C06F010EC16FF350D4
:10603C000001C027F4500001C123C0C060F0C1C0F2
:10604C0061F00001C3C062F00001636B000E00013F
:10605C00656F060E0001646FE8EC18F000016151E9
:10606C0000016011D8B410D00001FD51010D0101E7
:10607C00D00EF324D96E0101010EF420DA6E00016A
:10608C00C3C0DFFF0001FD2B0001C52B050E000175
:10609C00C565A9D70FD00001FD51010D0101D00E2E
:1060AC00F324D96E0101010EF420DA6E0E0EDF6EB0
:1060BC000001FD2B0001FD51800A780FD8A0EBD711
:1060CC000001EEA502D00101D1810101010E0001F8
:1060DC00616F0101D00E0001606F0101010E000122
:1060EC00636F0101960E0001626F000E0001656F77
:1060FC00080E0001646F20EC19F0000161510001E1
:10610C006011D8B47BD00101010E0001616F010157
:10611C00D20E0001606F0101010E0001636F0101DD
:10612C00980E0001626F000E0001656F060E0001F3
:10613C00646F20EC19F00001615100016011D8A4CA
:10614C000FD00101D2510E0AD8B40AD00101D16787
:10615C0007D0D0C1C0F0220E0001C017D8B420D097
:10616C000101D2510E0AD8B402D0000E4E6E0101BC
:10617C00010E0001AD6F0101D00E0001AC6F0101E9
:10618C00010E0001AF6F0101960E0001AE6F000110
:10619C00BFC0B1F00001BEC0B0F055EC31F02CD056
:1061AC0001019751D8B404D00101D151D8B426D0F3
:1061BC00010196A303D00101D0A320D0010196AB1D
:1061CC0003D00101D0AB1AD00101010E0001AD6F5B
:1061DC000101D00E0001AC6F0101010E0001AF6F87
:1061EC000101960E0001AE6F0001BFC0B1F00001BD
:1061FC00BEC0B0F055EC31F00001C26F0001BFC061
:10620C006DF00001BEC06CF0B1EC2DF033D000018C
:10621C00EB51040F0001C66F040E0001C66503D0DC
:10622C00050E0001C65F0001EB51060D0101A60E23
:10623C00F3240001606F0101010EF4200001616F75
:10624C000001C651060DA60E0001C06F010EC16FF4
:10625C00F3500001C027F4500001C123C0C062F00C
:10626C00C1C063F0000E0001656F060E0001646F83
:10627C00D6EC22F00001EB2B040E0001EB6503D0F1
:10628C00000E0001EB6F020E0001FD6F000E00010D
:10629C00FB6F000E0101D16F0001C2511200000111
:1062AC00ADC061F00001ACC060F00001AFC063F0A4
:1062BC000001AEC062F0000E0001656F080E000117
:1062CC00646F20EC19F00001615100016011D8A439
:1062DC0002D0000EBDD10001B1C061F00001B0C010
:1062EC0060F0000E0001636F000E0001626F000E83
:1062FC000001656F080E0001646F1EEC15F00001C3
:10630C0020EE01F00001AC51D9260001AD51DA228A
:10631C00DF500001B26F0001B2A133D1ACC0D9FF84
:10632C00ADC0DAFFDF500001B66F020E0001B86F8E
:10633C00010E0001BC6F020E0001B96F10D10001FB
:10634C00B951010DF3500001AC25D96EF450000188
:10635C00AD21DA6EDF500001B76F0001B751CBEC05
:10636C0023F000016EC0B4F000016FC0B5F0000E58
:10637C000001BA6FE9D00001BA51010D0001B4C09F
:10638C00B2F00001B5C0B3F0F3500001B227F450E5
:10639C000001B323B2C0F6FFB3C0F7FF0800000141
:1063AC00F5CFBBF0020E0001AE250001606F000EB0
:1063BC000001AF210001616F0001B7C062F0000164
:1063CC00636B000E0001656F060E0001646FE8EC54
:1063DC0018F00001615100016011D8A402D0010E27
:1063EC0001D0000E0001BD6F80D00001BD51D8B4AA
:1063FC00A9D0EDEC25F037D00001BD51D8B4A2D016
:10640C0084EC14F030D00001BD51D8B49BD0F4EC26
:10641C0013F029D00001BD51D8B494D03CEC14F049
:10642C0022D00001BD51D8B48DD00CEC14F01BD08F
:10643C000001BD51D8B486D06CEC14F014D000011E
:10644C00BD51D8B47FD024EC14F00DD00001BD5157
:10645C00D8B478D054EC14F006D00001BD51D8B4A7
:10646C0071D09CEC14F0040E0001BC6F6BD00001D9
:10647C00B68168D0110E0001B61364D00001B6834A
:10648C0061D00001B68B5ED00001BB51900AD8A43C
:10649C0002D0010E06D00001BB51910AD8A404D041
:1064AC00000E0001ED6F10D00001BB51390AD8A4C9
:1064BC000BD00001BD51D8B407D08AEC13F0000901
:1064CC00D8B402D0010E471A0001B851010DF35097
:1064DC000001B025D96EF4500001B121DA6E000133
:1064EC00BBC0DFFF0001B82B2DD00001BB51000A4F
:1064FC00D8B428D03A0AD8B478D7010AD8B47CD703
:10650C00070AD8B480D7010AD8B484D7030AD8B400
:10651C0088D7010AD8B48CD77F0AD8B490D7010A8F
:10652C00D8B494D7030AD8B498D7A20AD8B49FD7B2
:10653C00010AD8B4A3D7050AD8B49CD7010AD8B499
:10654C00A0D7A2D70001BA2B030E0001BA5DD8B0B8
:10655C0004D0070E0001B8650ED70001B92B080E48
:10656C000001B95DD8B005D00001BC51040AD8A413
:10657C00E6D6B0C0D9FFB1C0DAFF0001B6C0DFFF6C
:10658C0043D00001ADC061F00001ACC060F03AEC4A
:10659C0015F00009D8B422D04750D8B40AD0000165
:1065AC00F351040AD8B41AD00001F351050AD8B437
:1065BC0015D00001ADC0A7F00001ACC0A6F00001E1
:1065CC00AFC0A9F00001AEC0A8F00001B1C0ABF0A3
:1065DC000001B0C0AAF05FEC2AF014D00001ADC0ED
:1065EC0079F00001ACC078F00001AFC07BF0000185
:1065FC00AEC07AF00001B1C07DF00001B0C07CF0FB
:10660C005BEC28F00001BC6F0001BC05D8B40AD0CB
:10661C000001BC51030AD8B405D00001BC51040AD6
:10662C00D8A414D00001AFC061F00001AEC060F07E
:10663C000001ADC063F00001ACC062F0000E0001BF
:10664C00656F080E0001646FD6EC22F00001BC519E
:10665C0012000001FC51020AD8B436D00001FC51E2
:10666C00030AD8B431D00101A4C1C7F00101A5C1FE
:10667C00C8F00001C71FC81FC74BC82BB4EC12F0E1
:10668C000001C751000160270001C85100016123BE
:10669C0000016151800A800F8D0ED8B40001605D3D
:1066AC00D8A0E1D7B4EC12F0000160C0A4F1000155
:1066BC0061C0A5F13D2A3DC0C7F00001C86BC7BF42
:1066CC00C8070001C7B1A7D101019F519E11D8B4D1
:1066DC0013D09EC1D9FF9FC1DAFFDFAE04D00001F9
:1066EC00C76BC72B02D00001C76B0001C75100015B
:1066FC00CA6F0001CB6B06D0000E0001CB6F000EF1
:10670C000001CA6F0001CB51CA11D8A44AD10001B3
:10671C00FC51030AD8A419D005010251D8B40AD0EF
:10672C00B2EC13F005010219D8A404D0000E050137
:10673C00026F1CD178EC16F00501026F050102679F
:10674C0015D1000E0001FC6F11D1070E0001D06FA6
:10675C0082D00001D051010D01017C0EF324D96EC1
:10676C000101010EF420DA6EDF50FF0A0001C76F41
:10677C000001D051020D0101300EF324D96E01013C
:10678C00010EF420DA6EDECFC8F0DDCFC9F0C8C040
:10679C00D9FFC9C0DAFF0001C751DF16000E000196
:1067AC00CF6F2FD00001CF51010D0101500EF324FA
:1067BC00D96E0101010EF420DA6EDF500001C76FB3
:1067CC000001CF51020D0101000EF324D96E01011D
:1067DC00010EF420DA6EDECFC8F0DDCFC9F0C8C0F0
:1067EC00D9FFC9C0DAFFDF500001C7150009D8A4D2
:1067FC0006D0CFC078F00001D05120EC27F000017A
:10680C00CF2B0B0E0001CF65CDD70001D051010D60
:10681C0001017C0EF324D96E0101010EF420DA6E15
:10682C00DF500001C76F0001D051020D0101300E85
:10683C00F324D96E0101010EF420DA6EDECFC8F01C
:10684C00DDCFC9F0C8C0D9FFC9C0DAFF0001C751FC
:10685C00DF120001D0070001D0AF7BD70501050E78
:10686C000001BF6F0501000E0001BE6F81EC2FF01F
:10687C000001FC6F6DD00501050E0001616F050173
:10688C00100E0001606F000E0001636F000E00011E
:10689C00626F000E0001656F060E0001646F1EEC46
:1068AC0015F064D0000E0001CE6F10D00001CE5157
:1068BC00010D0501020EF324D96E0501050EF4201D
:1068CC00DA6EDF5035EC17F00001CE2B050E00010F
:1068DC00CE65ECD7060EC6EC12F00501026F050171
:1068EC00050E0001616F0501030E0001606F000EC3
:1068FC000001636F000E0001626F000E0001656FF6
:10690C00050E0001646F1EEC15F030D0030E000173
:10691C00FC6F000E0501006F800EC6EC12F0050135
:10692C00026F0501050E0001616F0501030E0001E8
:10693C00606F000E0001636F000E0001626F000EAD
:10694C000001656F050E0001646F1EEC15F00ED092
:10695C000001FC51010AD8B409D0030AD8B48BD772
:10696C00010AD8B49FD7070AD8B4D0D70001FC517C
:10697C00D8B417D0010E0001606F0501050E00019F
:10698C00626F0501000E0001616F080E0001636F5C
:10699C00010E4FEC23F0000160C09EF1000161C0BC
:1069AC009FF10101A151A011D8B413D0A0C1D9FFFE
:1069BC00A1C1DAFFDFAE04D00001C76BC72B02D038
:1069CC000001C76B0001C7510001CC6F0001CD6BFA
:1069DC0006D0000E0001CD6F000E0001CC6F00013F
:1069EC00CD51CC11D8A417D0000E0001606F050159
:1069FC00050E0001626F0501080E0001616F010EAA
:106A0C000001636F010E4FEC23F0000160C0A0F198
:106A1C00000161C0A1F112000001826FA10E000102
:106A2C00825DD8B098D0000182C060F00001616B2B
:106A3C00000E0001636F070E0001626F0FEC20F077
:106A4C00D8900001603700016137520E00016025BB
:106A5C0000017F6F7D0E000161210001806F000E2F
:106A6C000001816F23D000018151010D00017FC015
:106A7C007AF0000180C07BF0F35000017A27F450CB
:106A8C0000017B237AC0F6FF7BC0F7FF0001815128
:106A9C00010DF35000017825D96EF45000017921D5
:106AAC00DA6E0800F5CFDFFF0001812B020E00012A
:106ABC00815DD8B018D000018151010D00017FC05B
:106ACC007AF0000180C07BF0F35000017A27F4507B
:106ADC0000017B237AC0F6FF7BC0F7FF0800F5505E
:106AEC000009D8A4C0D7000182C060F00001616B1E
:106AFC00000E0001636F070E0001626F3EEC1DF08B
:106B0C007B0E00016025F66E770E00016121F76E99
:106B1C0000018151010DF35000017825D96EF4501C
:106B2C0000017921DA6E0800F5CFDFFF0DD00001EE
:106B3C008151010DF35000017825D96EF4500001FC
:106B4C007921DA6E000EDF6E0001812B020E00013E
:106B5C008165EDD75ED1A00E000182652FD0B70EF6
:106B6C000001825DD8B02AD0000179C06FF000011D
:106B7C0078C06EF05F0E000182250001686F000185
:106B8C00696BFF0E6923000E00016B6F030E000191
:106B9C006A6FE7EC14F09E0E000168250001706F1F
:106BAC007C0E000169210001716F000E0001736FF2
:106BBC00030E0001726F47EC18F02BD1C70E0001C9
:106BCC0082653FD0E10E0001825DD8B03AD0000161
:106BDC0079C06FF0000178C06EF0700E00017A6F12
:106BEC00FE0E7B6F0001825100017C6F7D6BD89093
:106BFC0000017C377D3700017A5100017C270001B0
:106C0C007B5100017D23200E00017C250001706F5B
:106C1C007D0E00017D210001716F000E0001736F6C
:106C2C00020E0001726F47EC18F0000120EE02F02A
:106C3C0000017851D92600017951DA22000EDF6E5D
:106C4C00E8D0E50E00018265D0D0F20E0001825D25
:106C5C00D8A065D0CAD01A0E000182250001686F39
:106C6C000001696BFF0E6923000E00016B6F030EB0
:106C7C0000016A6FE7EC14F0930E00016825000127
:106C8C007F6F7E0E47D01A0E000182250001686FBF
:106C9C000001696BFF0E6923000E00016B6F030E80
:106CAC0000016A6FE7EC14F04B0E0001682500013F
:106CBC007F6F7E0E2FD01A0E000182250001686FA7
:106CCC000001696BFF0E6923000E00016B6F030E50
:106CDC0000016A6FE7EC14F06F0E000168250001EB
:106CEC007F6F7E0E17D01A0E000182250001686F8F
:106CFC000001696BFF0E6923000E00016B6F030E20
:106D0C0000016A6FE7EC14F0FF0E0001682500012A
:106D1C007F6F7E0E000169210001806F0FD0000192
:106D2C00EC51000AD8B4DFD7010AD8B4C4D7030A8F
:106D3C00D8B491D7010AD8B4A6D7D5D7000E000184
:106D4C00816F020E0001816501D063D00001815179
:106D5C00010D00017FC07AF0000180C07BF0F35080
:106D6C0000017A27F45000017B237AC0F6FF7BC028
:106D7C00F7FF08000001F5CF7EF08AEC13F0000954
:106D8C00D8A40DD01DD0300E07D0320E05D02E0E4B
:106D9C0003D0250E01D0260E00017E6F11D000010C
:106DAC007E51260AD8B4F5D7010AD8B4F4D7080A0C
:106DBC00D8B4E9D71F0AD8B4E8D7050AD8B4E7D7AE
:106DCC0000018151010DF35000017825D96EF4506A
:106DDC0000017921DA6E00017EC0DFFF0001812BFA
:106DEC00020E00018165B2D714D0000179C061F0A8
:106DFC00000178C060F0000E0001636F000E00010E
:106E0C00626F000E0001656F030E0001646F1EECD3
:106E1C0015F0120083C0D9FF84C0DAFFDF500001E7
:106E2C00A06F020E0001A56F010E0001916F83C0CF
:106E3C00D9FF84C0DAFFDF50DD0B0001976F87C0EC
:106E4C00D9FF88C0DAFF000197C0DFFF020E0001F6
:106E5C00966F0BD300019651010DF3500001832561
:106E6C00D96EF45000018421DA6EDF500001A16F5D
:106E7C000001A1C060F00001616B000E0001636FA6
:106E8C000C0E0001626F0FEC20F00001605100014C
:106E9C00A36F0001A1C060F00001616B000E000146
:106EAC00636F0C0E0001626F3EEC1DF0000160512F
:106EBC000001A26F0001A15126EC1CF00001A46F8F
:106ECC000001A451D8B425D00001A551010DF350F7
:106EDC0000018725D96EF45000018821DA6E00017B
:106EEC00A4C0DFFF0001A52B000E0001616F4F0E47
:106EFC000001606F000E0001636F000E0001626FF5
:106F0C00000E0001656F030E0001646F1EEC15F09E
:106F1C0032D1000E0001926F030E0001A36512D056
:106F2C00070E0001A35DD8B00DD00001A251050AD7
:106F3C00D8B408D00001A251060AD8B403D0010E6F
:106F4C000001926F92C095F0020E0001986F1FD055
:106F5C0000019551D8B419D000019851010DF3508E
:106F6C0000018525D96EF45000018621DA6E0001EE
:106F7C00A151DF620AD00E0E0001A16F010E0001BB
:106F8C00A36F020E0001A26F06D00001982B070E12
:106F9C0000019865DDD7A0C08FF0220E00018F177D
:106FAC0000018F51220AD8A411D04AA203D00001AB
:106FBC00A0930CD085C0D9FF86C0DAFFDF5000014A
:106FCC008F6F00018FAB02D00001A09B060E000159
:106FDC00A36504D0000E00019F6F3AD00001A0A35E
:106FEC000AD00001A3510C0D00018BC08FF00001E1
:106FFC008CC090F016D00001A0AB0AD00001A351B8
:10700C000C0D00018DC08FF000018EC090F009D0E6
:10701C000001A3510C0D000189C08FF000018AC042
:10702C0090F0F35000018F27F450000190230001E1
:10703C00A251010DF35000018F27F4500001902351
:10704C008FC0F6FF90C0F7FF08000001F5CF9FF04E
:10705C0000019F51D8B40CD00001000E0001796FD3
:10706C0000019C0E0001786F00019F5112EC35F06D
:10707C0000019F51D8B403D000019C678AD0000155
:10708C00A151CDEC24F00001A46F0001A451D8B49F
:10709C00EAD10001A451900AD8A402D0010E06D066
:1070AC000001A451910AD8A404D0000E0001ED6F88
:1070BC003ED00001A451390AD8A425D0020E0001FB
:1070CC0085250001606F000E000186210001616FB3
:1070DC000001A4C062F00001636B000E0001656F3B
:1070EC00060E0001646FE8EC18F00001615100011C
:1070FC006011D8A41CD08AEC13F00009D8B417D0B6
:10710C00010E471A14D00001A451270AD8A40FD09D
:10711C00A0C08FF0220E00018F17D8B408D08AECD3
:10712C0013F00009D8B403D0870E0001A46F00013E
:10713C00A551010DF35000018725D96EF4500001C3
:10714C008821DA6E0001A4C0DFFF0001A52B000E20
:10715C000001616F4F0E0001606F000E0001636F44
:10716C00000E0001626F000E0001656F030E00013E
:10717C00646F1EEC15F083C0D9FF84C0DAFFDF50BA
:10718C004A6E83C0D9FF84C0DAFFDF500001976FCD
:10719C006AD100019551D8B463D0000E0001996FEB
:1071AC004CD0000E00019A6F33D000019951010DA3
:1071BC000101E00EF324D96E0101010EF420DA6E08
:1071CC0000019A51010D00019C0EF324E16E0001A7
:1071DC00000EF420E26EE750DF6218D00101010EC0
:1071EC000001616F0101E00E0001606F000E0001F3
:1071FC00636F000E0001626F000E0001656F030EDD
:10720C000001646F1EEC15F0020E7CD100019A2B6C
:10721C00030E00019A5DD8B00ED000019A51010DF9
:10722C0000019C0EF324D96E0001000EF420DA6EDE
:10723C00DF50D8A4BAD70001992B030E0001995D39
:10724C00D8B00ED000019951010D0101E00EF324CC
:10725C00D96E0101010EF420DA6EDF50D8A4A1D74B
:10726C00030E0001916F000E00019B6FC9D000014D
:10727C009B51010D00019C0EF324D96E0001000EF0
:10728C00F420DA6EDF500001A46FA9D04F50D8B4AF
:10729C00B5D07F0E0001616FF60E0001606F00012A
:1072AC004FC062F00001636B000E0001656F040EAD
:1072BC000001646FE8EC18F0000160C093F000016D
:1072CC0061C094F0000194519311D8B497D0060E7C
:1072DC000001A55DD8B092D00001A551010DF3506D
:1072EC0000018725D96EF45000018821DA6E2A0E30
:1072FC00DF6E0001A52BF60E00018F6F7F0E906FD5
:10730C0000018F1F901F8F4B902B00019351000198
:10731C008F270001945100019023880E00018F25C6
:10732C00F66E770E9021F76E0001A551010DF3500A
:10733C0000018725D96EF45000018821DA6E08000F
:10734C00F5CFDFFF25D04F500B0AD8A457D0060E2F
:10735C000001A55DD8B052D00001A551010DF3502C
:10736C0000018725D96EF45000018821DA6E2A0EAF
:10737C00DF6E0001A52B0001A551010DF35000019A
:10738C008725D96EF45000018821DA6E130EDF6E5A
:10739C000001A52B0001A551010DF350000187251B
:1073AC00D96EF45000018821DA6E50C0DFFF14D082
:1073BC000001978323D00001978B20D00001A551A9
:1073CC00010DF35000018725D96EF450000188217E
:1073DC00DA6E0001A4C0DFFF0001A52B0FD0000165
:1073EC00A451E10AD8B4E4D7040AD8B4E4D7160AF5
:1073FC00D8B44CD7070AD8B4A6D7E0D700019B2B3A
:10740C00030E00019B5DD8B012D000019B51010D01
:10741C0000019C0EF324D96E0001000EF420DA6EEC
:10742C00DF50D8B404D0070E0001A56520D7000E9C
:10743C0000016F6F4F0E00016E6F0001000E000116
:10744C00716F00019C0E0001706F000E0001736FD4
:10745C00030E0001726F47EC18F083C0D9FF84C093
:10746C00DAFFDF504A6E0001962B080E0001965D84
:10747C00D8B004D0070E0001A565ECD4020E0001B3
:10748C00A5651ED00101010E00016F6F0101E00E18
:10749C0000016E6F000E0001716F4F0E0001706FD6
:1074AC00000E0001736F030E0001726F47EC18F0B1
:1074BC0087C0D9FF88C0DAFF000197C0DFFF20D05A
:1074CC000101010E0001616F0101E00E0001606F0E
:1074DC00000E0001636F000E0001626F000E0001D0
:1074EC00656F030E0001646F1EEC15F083C0D9FFAD
:1074FC0084C0DAFF87C0E1FF88C0E2FFDFCFE7FF7F
:10750C00000191511200000D010203040506070849
:10751C00090A1624000E0E0E0E0E0E0E0E0B2F5414
:10752C00180E0E0E41420E0E0E235F550C0E0E0E53
:10753C004D4E0E0E0E175E5619252627282B2C2D78
:10754C002E225D5730313233343738393A3B5C5860
:10755C003C3D3E3F4043444546475B5948494A4BB6
:10756C004C4F505152535A2F3B3C3D3E3F404142B1
:10757C0043442E353A000000000000000045313035
:10758C001E0000000000000000272D2A1F202122D1
:10759C0000002324252634141A09130A00000D0FA9
:1075AC00181C33041516170729650B11080C121D2E
:1075BC001B0619052B280E10363738E0E3F0E12CAA
:1075CC00E2E62CE5F0E7E42F3B3C3D3E3F404142F8
:1075DC00434431353A0000000000000000452E30D5
:1075EC001E00000000000000002738391F20212257
:1075FC000000232425262D343637131C0000090ADD
:10760C0006150F041208180C2965070B17111633F1
:10761C00140D0E1B2B2805101A191DE0E3F0E12A9E
:10762C00E2E62CE5F0E7E4303B3C3D3E3F40414296
:10763C0043442E893A0000000000000000452F3220
:10764C001E0000000000000000272D391F20212201
:10765C0000002324252634141A08151700001C18C2
:10766C000C1213041607090A29650B0D0E0F331D96
:10767C001B0619052B281110363738E0E3F0E12AE8
:10768C00E2E62CE5F0E7E4303B3C3D3E3F40414236
:10769C0043442D893A0000000000000000452F32C1
:1076AC001E000000000000000027342E1F202122A5
:1076BC000000232425262A141A08151700001C186C
:1076CC000C1213041607090A29650B0D0E0F331D36
:1076DC001B0619052B281110363738E0E3F0E1585A
:1076EC00E2E62CE5F0E7E42F3B3C3D3E3F404142D7
:1076FC0043442E353A0000000000000000453130B4
:10770C001E0000000000000000272D391F20212240
:10771C0000002324252634141A08151700001C1801
:10772C000C1213041607090A29650B0D0E0F331DD5
:10773C001B0619052B281110363738E0E3F0E12A27
:10774C00E2E62CE5F0E7E400000000000000000099
:10775C00000000005500FB00675400005F6061569C
:10776C00005C5D5E5700595A5B28006200630000A4
:10777C00040C1808121CFA7F3F7FAA7D0A1D07050E
:10778C00D47D4900003B00003C00003D00003E0061
:10779C00003F00004000004100004200007F00005C
:1077AC00810000480000E04C003A0000000000009E
:1077BC0000000000000000000000000000000000BD
:1077CC0000000000800000470000E0E11DE01E000A
:1077DC00000000000000000000000000000000009D
:1077EC000000000000000000E027004600004C00F4
:1077FC0000E01F00E02000E02100E022000000007B
:10780C00000000E02300E0E150E15200E0E14F53C2
:10781C000000E01400E01A004B0000E01500E01737
:10782C0000000000000000E04A00E05000520000A0
:10783C00E04F00E04D00E00400E016004E0000E0D8
:10784C000900E00A002900003900004A000050003D
:10785C00005100004F00004D0000E01D00E01B0037
:10786C00E00600E019009100002B000028000090B9
:10787C000000E15000E15100E14F00E14D0000003B
:10788C0000000000000000000000E02A00000000E2
:10789C00000000E02C0000000000000000000000D0
:1078AC0000000000000000000000000000000000CC
:1078BC0000000000000000000000000000000000BC
:1078CC0000000000000000000000000000000000AC
:1078DC000000B69AB5B4B300002A31383F46040311
:1078EC000201050000070E151C23AE6993A4B2001B
:1078FC00004D545BCD620000000000000000000051
:10790C00000000000000000000000000000000006B
:10791C00000000000000000000000000000000005B
:10792C00000000000000ACA9A6A2B00000307A3E16
:10793C00C84CABA8A5A1AF00000D141B2229ADAA01
:10794C00A7A3B10000535A61CE68000000000000EC
:10795C000000000000CA0000000000000000000051
:10796C0000000000000000000000000000CD00003E
:10797C0000000000000000000000CE08160C0F00F4
:10798C000039170A18CD0310190B120000241A091C
:10799C0002C8CE2511262700002E132028EC00004B
:1079AC00000000000000000000CA00000000000001
:1079BC0000000000000000CC0000000000000000EF
:1079CC00000000EDF1E6E70000EAEB0000006A04BD
:1079DC003A7F3C0000475D505E4844011D812F00FA
:1079EC000063604F4BC86CC93D326B000049594A6B
:1079FC0067ECE800000000000000000000CB000075
:107A0C0000000000000000000000E9CC00000000B5
:107A1C0000000000000000EDF1E6E70000EAEB00DA
:107A2C000000CE4E5C52550000361E3B2B6D965618
:107A3C005F515800002C0521837ACE64576566008F
:107A4C00001F342D406ED300000000000000000029
:107A5C000000000000000000000000000000D4D76F
:107A6C00000000000000000000DE0000000000002C
:107A7C000000000000DD000000000000000000001D
:107A8C0000D1000000000000000000000000000019
:107A9C00DB0000000000000000E0D300000000004C
:107AAC0000000000000000000000000000000000CA
:107ABC000000D400000000000000000000DE000008
:107ACC00000000000000000000DF000000B3000018
:107ADC000000000000D2000046D6D5000000D9D826
:107AEC00DC000000000000000000DA0000000000D4
:107AFC00000000000000000000000000000000007A
:107B0C000000000000000000000000000000000069
:107B1C000000000000000000000000000000393BE5
:107B2C000C2483000009210A013C161A08192F00A5
:107B3C000044020310C82B3A1E0F1D00001118CD73
:107B4C00CE7A000000000000000000000000EE00F3
:107B5C000000000000000000000000000000000019
:107B6C000000000000000000000000000000000009
:107B7C0000002513EC7F2800004F5150CC8E1F20A5
:107B8C008136260000CA5D9656906D6E1234270021
:107B9C0000575EEFF086E8000000000000000000D7
:107BAC000000000000000000000000000000E900E0
:107BBC0000000000000000000000000000000000B9
:107BCC0000000000000064595263670000040B2E93
:107BDC002D3D5C604E5F6500000517C92C32717439
:107BEC005855660000406B6ACB6C0000000000002A
:107BFC000000000000000000000000000000000079
:107C0C000000000000000000000000000017000051
:107C1C000000000000000000001D130B121983006F
:107C2C000018C821443A2408101A1600000A03024E
:107C3C00CA09110C1E0F0100007A3BCDCE3CE800A6
:107C4C000000000000000000000000000000000028
:107C5C00000000000000E90000000000000000002F
:107C6C0000E60000000000000000000000E76ACB06
:107C7C0028262E000025042C321F6B273981360054
:107C8C00002B052F40346C6D6E207F00002D3DECD9
:107C9C00C9CC041111040E18041718040C000C1193
:107CAC00110C0E180C1718181111180E181817188B
:107CBC00081111080E0C081718080C0012111112DB
:107CCC000E181217181218000600000900000D00FB
:107CDC000014000005010906A101050719E029E7B8
:107CEC001500250175019508810295017508810320
:107CFC009505750105081901290591029501750372
:107D0C00910395067508150026FF00050719002933
:107D1C00FF8100C011112D00F300F400E138360092
:107D2C003700E136E1372F003000E130E13234002A
:107D3C002E002D001E0038003200E1278700E136AE
:107D4C00E137E138890000000E0016001700110021
:107D5C000B0010001C0015001A0013000A001D0077
:107D6C00070005001B001B0E1B171B1C1B1A1A1CE3
:107D7C0019000F00E0E1E3E2E6E5E4E0E1E29190D6
:107D8C00E5E4E0E1E39190E5E4E1E0E3E2E6E4E55B
:107D9C00E1E0E29190E4E5E1E0E39190E4E52A038F
:107DAC0045007300720069006C006C0065002000D7
:107DBC004E006500770020004B00650079006200E2
:107DCC006F0061007200640009022900010100A02B
:107DDC003209040000020301010009211101000114
:107DEC002240000705810308000107050103080074
:107DFC0001130628000010040628001E2721042861
:107E0C001E272105281E272604281E2726052804A0
:107E1C002D161328162D1613280612131C150C0AD2
:107E2C000B172C1F271E20362C1F271E212C081643
:107E3C00150C0F0F082C0C11063728091F2C002FBE
:107E4C000000300000E12F00E13000E2E126E2E129
:107E5C00273800003800003838383600003700006A
:107E6C00E135002F00003000002F00003000002F03
:107E7C000000300000380000380000383838360078
:107E8C0000370000E135002F00003000001D2F00EE
:107E9C001D30002F00003000001D38003800001D80
:107EAC003700360000370000E135001512100428A9
:107EBC0000110C0612280010171C13082817151295
:107ECC0011280016170C060E281B2327272128061D
:107EDC002800000000060D28000000060D10040606
:107EEC0028162800000000160D28000000160D10A2
:107EFC000406282F00003000002F00003000002F57
:107F0C0000003000003800003800003838383600E7
:107F1C0000370000E135000F28000006280000158E
:107F2C002800000F2D1128062D0628152D162812B5
:107F3C000909281A0345007300720069006C006C73
:107F4C00006500200049006E0063002E0018162802
:107F5C00000018162D072818162D06280D132800BA
:107F6C00000D132D11280816150C0F0F082C110CD1
:107F7C0016160828150819372C0007272800071E85
:107F8C001F28071F21280720232807212528101622
:107F9C002800000417120E280A12120A28041313C0
:107FAC000F281201000200000008D80450F501004F
:107FBC00010200018B00008A0000880000350000DF
:107FCC001209092812112800190815372C00092646
:107FDC002C0009202C0009212C0009222C0009233B
:107FEC002C0009242C0009252C000E16170B040359
:047FFC000904000074
:020000040020DA
:08000000FFFFFFFFFFFFFFFF00
:020000040030CA
:0E000000330E3F1EFF8181FF0FC00FE00F4047
:0200000400F00A
:080000000000000100040000F3
:00000001FF
